BL51 BANKED LINKER/LOCATER V4.13                                                        12/01/2007  15:27:31  PAGE 1


BL51 BANKED LINKER/LOCATER V4.13, INVOKED BY:
C:\KEIL\C51\BIN\BL51.EXE STARTUP.obj, Text1.obj TO LED_A RAMSIZE (256)


INPUT MODULES INCLUDED:
  STARTUP.obj (?C_STARTUP)
  Text1.obj (TEXT1)


LINK MAP OF MODULE:  LED_A (?C_STARTUP)


            TYPE    BASE      LENGTH    RELOCATION   SEGMENT NAME
            -----------------------------------------------------

            * * * * * * *   D A T A   M E M O R Y   * * * * * * *
            REG     0000H     0008H     ABSOLUTE     "REG BANK 0"
            IDATA   0008H     0001H     UNIT         ?STACK

            * * * * * * *   C O D E   M E M O R Y   * * * * * * *
            CODE    0000H     0003H     ABSOLUTE     
* OVERLAP * CODE    0000H     004AH     ABSOLUTE     
            CODE    004AH     000FH     UNIT         ?C_C51STARTUP



UNRESOLVED EXTERNAL SYMBOLS:
   ?B_SWITCH0
   ?C_START



SYMBOL TABLE OF MODULE:  LED_A (?C_STARTUP)

  VALUE           TYPE          NAME
  ----------------------------------

  -------         MODULE        ?C_STARTUP
  C:004AH         SEGMENT       ?C_C51STARTUP
  I:0008H         SEGMENT       ?STACK
  C:0000H         PUBLIC        ?C_STARTUP
  N:0000H         SYMBOL        IBPSTACK
  N:0100H         SYMBOL        IBPSTACKTOP
  N:0080H         SYMBOL        IDATALEN
  C:004DH         SYMBOL        IDATALOOP
  N:0000H         SYMBOL        PBPSTACK
  N:0000H         SYMBOL        PBPSTACKTOP
  N:0000H         SYMBOL        PDATALEN
  N:0000H         SYMBOL        PDATASTART
  N:0000H         SYMBOL        PPAGE
  N:0000H         SYMBOL        PPAGEENABLE
  D:0081H         SYMBOL        SP
  C:004AH         SYMBOL        STARTUP1
  N:0000H         SYMBOL        XBPSTACK
  N:0000H         SYMBOL        XBPSTACKTOP
  N:0000H         SYMBOL        XDATALEN
  N:0000H         SYMBOL        XDATASTART
  C:0000H         LINE#         80
BL51 BANKED LINKER/LOCATER V4.13                                                      12/01/2007  15:27:31  PAGE 2


  C:004AH         LINE#         87
  C:004CH         LINE#         88
  C:004DH         LINE#         89
  C:004EH         LINE#         90
  C:0050H         LINE#         139
  C:0053H         LINE#         141
  C:0056H         LINE#         142
  -------         ENDMOD        ?C_STARTUP

  -------         MODULE        TEXT1
  C:003FH         SYMBOL        D0
  C:0041H         SYMBOL        D1
  C:0043H         SYMBOL        D2
  C:003DH         SYMBOL        DELAY
  B:0090H.0       SYMBOL        LED
  D:0090H         SYMBOL        P1
  C:0030H         SYMBOL        START
  C:0000H         LINE#         13
  C:0030H         LINE#         17
  C:0032H         LINE#         18
  C:0035H         LINE#         19
  C:0037H         LINE#         20
  C:003AH         LINE#         21
  C:003DH         LINE#         23
  C:003FH         LINE#         24
  C:0041H         LINE#         25
  C:0043H         LINE#         26
  C:0045H         LINE#         27
  C:0047H         LINE#         28
  C:0049H         LINE#         29
  -------         ENDMOD        TEXT1

*** WARNING L5: CODE SPACE MEMORY OVERLAP
    FROM:    0000H
    TO:      0002H

*** WARNING L1: UNRESOLVED EXTERNAL SYMBOL
    SYMBOL:  ?C_START
    MODULE:  STARTUP.obj (?C_STARTUP)

*** WARNING L1: UNRESOLVED EXTERNAL SYMBOL
    SYMBOL:  ?B_SWITCH0
    MODULE:  STARTUP.obj (?C_STARTUP)

*** WARNING L2: REFERENCE MADE TO UNRESOLVED EXTERNAL
    SYMBOL:  ?B_SWITCH0
    MODULE:  STARTUP.obj (?C_STARTUP)
    ADDRESS: 0054H

*** WARNING L2: REFERENCE MADE TO UNRESOLVED EXTERNAL
    SYMBOL:  ?C_START
    MODULE:  STARTUP.obj (?C_STARTUP)
    ADDRESS: 0057H

LINK/LOCATE RUN COMPLETE.  5 WARNING(S),  0 ERROR(S)
